:100000000C94AF030C94F6030C94F6030C94F603D3
:100010000C94F6030C94F6030C94F6030C94F6037C
:100020000C94F6030C94F6030C94831E0C94561F48
:100030000C9490150C94F6030C94F6030C94F603B0
:100040000C94F6030C94F6030C94F6030C94F6034C
:100050000C94F6030C94F1150C94F6030C94F6032F
:100060000C94F6030C94F6030C94F6030C94F6032C
:100070000C94F6030C94F6030C94F6030C94F6031C
:100080000C94F6030C94F6030C94F6030C94F6030C
:100090000C94F6030C94F6030C94F6030C94F603FC
:1000A0000C94F6030C94F6030C94F60301E2012B76
:1000B000022B00140008000000000012002F0000B6
:1000C000000000000000000400070009000E000FFF
:1000D000003400000000000000000029002800009B
:1000E000000000520050000000000000000000016D
:1000F000513E002C00000051004F000000000000A5
:10010000000000007001000000000001000100007C
:1001100000000000000000010001000100010001DA
:1001200000A8000000000000000000010001000025
:10013000000000AA00A9000000000000000000016B
:1001400000010001000000E2002B000000000000A0
:10015000000000010001000000000001000100009B
:10016000000000000000000100010001000100018A
:10017000000100000000000000000001000100007C
:10018000000000010001000000000000000000016C
:10019000000100010000000100010000000000005B
:1001A000000000010001000000000001000100004B
:1001B000000000000000000100010001000100013A
:1001C000000100000000000000000001000100002C
:1001D000000000010001000000000000000000011C
:1001E000000100010000000100010000000000000B
:1001F00000000001000100000000000100010000FB
:1002000000000000000000010001000100010001E9
:1002100000010000000000000000000100010000DB
:1002200000000001000100000000000000000001CB
:1002300000010001000000010001000000000000BA
:1002400000000001000100000000000100010000AA
:100250000000000000000001000100010001000199
:10026000000100000000000000000001000100008B
:10027000000000010001000000000000000000017B
:10028000000100010000000100010000000000006A
:10029000000000010001000000000001000100005A
:1002A0000000000000000001000100010001000149
:1002B000000100000000000000000001000100003B
:1002C000000000010001000000000000000000012B
:1002D000000100010000000100010000000000001A
:1002E000000000010001000000000001000100000A
:1002F00000000000000000010001000100010001F9
:1003000000010000000000000000000100010000EA
:1003100000000001000100000000000000000001DA
:1003200000010001000000010001000000000000C9
:1003300000000001000100000000000100010000B9
:1003400000000000000000010001000100010001A8
:10035000000100000000000000000001000100009A
:10036000000000010001000000000000000000018A
:100370000001000100000001000100000000000079
:100380000000000100010000000000010001000069
:100390000000000000000001000100010001000158
:1003A000000100000000000000000001000100004A
:1003B000000000010001000000000000000000013A
:1003C0000001000100000001000100000000000029
:1003D0000000000100010000000000010001000019
:1003E0000000000000000001000100010001000108
:1003F00000010000000000000000000100010000FA
:1004000000000001000100000000000000000001E9
:1004100000010001000000010001000000000000D8
:1004200000000001000100000000000100010000C8
:1004300000000000000000010001000100010001B7
:1004400000010000000000000000000100010000A9
:100450000000000100010000000000000000000199
:100460000001000100000001000100000000000088
:100470000000000100010000000000010001000078
:100480000000000000000001000100010001000167
:100490000001000000000000000000010001000059
:1004A0000000000100010000000000000000000149
:1004B0000001000100000001000100000000000038
:1004C0000000000100010000000000010001000028
:1004D0000000000000000001000100010001000117
:1004E0000001000000000000000000010001000009
:1004F00000000001000100000000000000000001F9
:1005000000010001000000010001000000000000E7
:1005100000000001000100000000000100010000D7
:1005200000000000000000010001000100010001C6
:1005300000010000000000000000000100010000B8
:1005400000000001000100000000000000000001A8
:100550000001000100000001000100000000000097
:100560000000000100010000000000010001000087
:100570000000000000000001000100010001000176
:100580000001000000000000000000010001000068
:100590000000000100010000000000000000000158
:1005A0000001000100000001000100000000000047
:1005B00000000012036B006500790062006F0061AB
:1005C00000720064000000160371006D006B006291
:1005D00000750069006C0064006500720000000492
:1005E00003090409026D00040100A0FA09040000D7
:1005F000010301010009211101000122400007054A
:10060000810308000A090401000103010200092115
:1006100011010001224D000705820308000A0904A8
:10062000020001030000000921110100012236002F
:100630000705830308000A09040300010300000002
:10064000092111010001223900070584032000015E
:100650001201100100000008EDFE606001000102BF
:10066000000105010906A101050719E029E71500A8
:1006700025019508750181020508190129059505CF
:10068000750191029501750391010507190029F77C
:100690001500250195F875018102C005010980A1A9
:1006A0000185021601002603001A81002A830075C5
:1006B0001095018100C0050C0901A10185031601F7
:1006C00000269C021A01002A9C02751095018100E7
:1006D000C005010902A1010901A1000509190129AB
:1006E00005150025019505750181029501750381A8
:1006F000010501093009311581257F9502750881B1
:100700000609381581257F950175088106050C0AB3
:1007100038021581257F950175088106C0C0050145
:100720000906A101050719E029E71500250195082B
:1007300075018102950175088101050819012905D6
:100740009505750191029501750391010507190041
:1007500029FF150026FF00950675088100C01124A9
:100760001FBECFEFDAE0DEBFCDBF04B603FE27C069
:100770008091290290912A02A0912B02B0912C0223
:100780008730904BA740B04BD1F4109229021092C1
:100790002A0210922B0210922C0214BE84B7877F7B
:1007A00084BF0FB6F894A89580916000886180930B
:1007B0006000109260000FBEE0E0F8E3099511E0E0
:1007C000A0E0B1E0E6E8F5E402C005900D92A633A2
:1007D000B107D9F722E0A6E3B1E001C01D92A9322A
:1007E000B207E1F70E94D91B0C9495220C940000EB
:1007F000FC01611106C08281882319F08CEA90E027
:10080000089590E080E008950895089581E00895A6
:10081000089581E008950C9406040E94E10D2FEFE5
:1008200084E39CE0215080409040E1F700C000004C
:100830000C941416EF92FF920F931F93CF93DF93B4
:100840008C01FC01E080F18080916A01811140C03F
:1008500082818823C1F1C7010E946613C82F682FC7
:10086000C7010E940F13B7018C2F0E945205EC01A3
:10087000B8010E940B04882309F44BC0B801CE01D3
:100880000E945B07882309F444C0C531F0E7DF0705
:1008900020F5C23080E7D80708F04DC0C115E0E769
:1008A000DE0791F1C130D047E1F181E0809338015A
:1008B00080933901C801DF91CF911F910F91FF9073
:1008C000EF900C940904C7010E943D13C82FCBCFB1
:1008D000C7010E946613B701C8CFCC3380E7D807A1
:1008E00009F49BC0CD33D04701F7F80182818823FA
:1008F00009F4BAC0109239010E94C01590933701D3
:100900008093360180E296C0F801828181110E94B5
:100910000D0480E0DF91CF911F910F91FF90EF9038
:100920000895F80182818823A1F38091E901816013
:100930008093E901EECFF8018281882309F4BACFD0
:100940000E942115811102C00E9407150E943E15C8
:1009500090E090931B0280931A02FE01E350F0474F
:1009600080911A028160E231F10538F4E956FD4DBB
:100970000C94452280911A02826080931A02809121
:100980001A020E9442150E94E10DC3CF80911A0203
:100990008460F3CF80911A028860EFCF80911A02B1
:1009A0008061EBCF80911A028062E7CF80911A02BA
:1009B0008064E3CF80911A028068DFCF80911A02B1
:1009C0008C60DBCF80911A028E7FD7CF80911A0284
:1009D0008D7FD3CF80911A028B7FCFCF80911A0267
:1009E000877FCBCF80911A028F7EC7CF80911A026A
:1009F0008F7DC3CF80911A028F7BBFCF80911A0267
:100A00008F77BBCF80911A02837FB7CF90911A0264
:100A1000892F97FB87F98058B0CFF801828188230E
:100A200061F0109238010E94C015909337018093B5
:100A3000360182E00E94460B6CCF80913801811113
:100A40000FC080913601909137010E94CC15883CEF
:100A5000910530F486E20E941B0A86E20E94F70AA2
:100A600082E00E944D0B55CF8091390181110FC05A
:100A700080913601909137010E94CC15883C9105F8
:100A800030F487E20E941B0A87E20E94F70A80E2A4
:100A9000E8CF0C94AA070C94AC070C9408040C94AF
:100AA0004D050895972F70E02AE0929F600D711D0B
:100AB0001124FB0198E2899FE00DF11D1124EE0F36
:100AC000FF1FED54FF4F859194910895FC01EE0FA7
:100AD000FF1FED54FA4F8591949108950E9452059D
:100AE0000E94DF069C01811540E4940708F097C03E
:100AF000211580E3380708F0FAC0203E310508F0E0
:100B000074C0203C310508F0E5C0283A310588F46E
:100B1000253A310508F0E2C02130310509F477C0EB
:100B2000C9010497813A910508F471C030E020E0D2
:100B30006EC0C901885A91094597C0F7283A310516
:100B400009F4FEC0293A310509F4FDC02A3A3105FD
:100B500009F4FCC02B3A310509F4FBC02C3A3105ED
:100B600009F4FAC02B3B310509F4F9C02C3B3105DF
:100B700009F4F8C02D3A310509F4F7C0203B3105DE
:100B800009F4F6C02E3A310509F4F5C02F3A3105C3
:100B900009F4F4C0213B310509F4F3C0223B3105CF
:100BA00009F4F2C0233B310509F4F1C0243B3105BF
:100BB00009F4F0C0253B310509F4EFC0263B3105AF
:100BC00009F4EEC0273B310509F4EDC0283B31059F
:100BD00009F4ECC0293B310509F4EBC02A3B31058F
:100BE00009F4EAC020E034E412C0211590E239078C
:100BF00080F42F3F310509F050F4283E310538F0DC
:100C0000C901805F91093065409708F08FCFC90115
:100C10000895C9019F700E9466059C01F8CF811557
:100C2000944508F041C0211583E5380708F06AC0F3
:100C3000211592E5390738F5211541E5340708F00B
:100C40005CC0211580E5380708F454C0C90134E0C0
:100C5000969587953A95E1F78370422F469546958C
:100C6000437090E2499FA0011124582B822F83707A
:100C700021E030E002C0220F331F8A95E2F7242BD7
:100C8000352B3C68C4CFC9018370992741E050E0FF
:100C900002C0440F551F8A95E2F72695269580E2FB
:100CA000289F90011124EBCF211596E5390748F4D0
:100CB000922F882721153545C8F59C01246F306A8D
:100CC000A6CFC90190563F708115904108F02ECFF4
:100CD00030629DCFC901805C91099DCF253A3105D5
:100CE00049F1263A310549F522E830E490CF33271F
:100CF000306C8DCF3F70306A8ACF322F2227216F20
:100D0000306A85CFC9018370992741E050E002C065
:100D1000440F551F8A95E2F72695269580E2289F75
:100D200090011124242B352B3A6871CF88279F71AD
:100D30009C01CECF21E830E46ACF23E830E467CFCE
:100D400022EE34E464CF29EE34E461CF2AEE34E4B9
:100D50005ECF25EB34E45BCF26EB34E458CF23EBB6
:100D600034E455CF24EB34E452CF27EB34E44FCFB7
:100D70002CEC34E44CCF2DEC34E449CF23E835E4BB
:100D800046CF2AE835E443CF22E935E440CF24E9D1
:100D900035E43DCF21E236E43ACF23E236E437CFE3
:100DA00024E236E434CF25E236E431CF26E236E4DD
:100DB0002ECF27E236E42BCF2AE236E428CF803E3E
:100DC000910581F1C8F48133910509F462C048F4BA
:100DD0008932910509F456C08A32910509F460C040
:100DE000089589339105B9F082389105A1F08533D2
:100DF000910509F440C00895863E910561F138F4EB
:100E0000823E9105B1F0833E9105E1F00895873E61
:100E1000910551F1089520911A022370D9F080EEC6
:100E200090E0089520911A0220FF14C089E390E019
:100E3000089520911A0222FF0DC024FD09C083EEFF
:100E400090E0089520911A0222FD31C024FF02C0D3
:100E500090E080E0089520911A0223FFFBCF24FD4B
:100E6000F7CF87EE90E0089520911A0223FFEECF8E
:100E700086EE90E0089520911A0225FFEBCF89E2DB
:100E800090E0089520911A0225FFE4CF85E390E0D9
:100E9000089520911A0226FFDDCF8AE290E008959E
:100EA00020911A0226FFD6CF81E390E0089582EECA
:100EB00090E0089508950F931F93CF938C01FB0149
:100EC0008281811106C0C1E08C2FCF911F910F91BB
:100ED0000895C0914701C11125C00531104799F708
:100EE0000E945A0781E0809347010E94C0159093A9
:100EF00046018093450110923A0110923C011092F4
:100F00003B0110923E0110923D011092400110925F
:100F10003F0110924201109241011092440110923F
:100F20004301D2CF80914501909146010E94CC159A
:100F3000883C910540F680913A01E82FF0E0EE0FF1
:100F4000FF1FE55CFE4F118300838F5F80933A01A2
:100F5000C0E0BACF0C9404040C940504CF93DF9343
:100F600085B7806885BF85B7806885BFADE1B1E092
:100F700041E251E0C1E0D0E08D91E82FE295EF70C1
:100F8000F0E061A18F709E0101C0220F8A95EAF7FF
:100F9000922F9095962391A382A1822B82A34A1728
:100FA0005B0751F7A3E1B1E04DE151E0C1E0D0E0D2
:100FB0008D91E82FE295EF70F0E061A18F709E01B6
:100FC00001C0220F8A95EAF7922F9095962391A35C
:100FD00082A1822B82A34A175B0751F7109251011D
:100FE0001092500110924901109248011092530141
:100FF0001092520110924B0110924A011092550129
:101000001092540110924D0110924C011092570110
:101010001092560110924F0110924E01DF91CF9124
:101020000C9449054F925F927F928F929F92AF925C
:10103000BF92CF92DF92EF92FF920F931F93CF93C5
:10104000DF9398E4492E91E0592E2DE1E22E21E024
:10105000F22E01E010E099249394E201A990B99056
:101060002E01DE011E921E92F70181917F01E82F71
:10107000E295EF70F0E091A18F70980101C0220F0E
:101080008A95EAF7892F822B81A382A1822E8094F0
:10109000882182A380EA8A95F1F783E1C82E81E056
:1010A000D82E90E080E0E60179916E01472F4295BD
:1010B0004F7050E0EA0178A04D915C9111977F70DC
:1010C000E80102C0CC0FDD1F7A95E2F7BE0167216F
:1010D00009F06AC0B801082E02C0660F771F0A9493
:1010E000E2F7462B572B11965C934E9301968A306C
:1010F0009105C9F681A1882281A282A1282B22A371
:101100008D919C91A816B90641F0909258010E94C9
:10111000C01590935A0180935901D0E54D16D1E046
:101120005D0609F09ACF80915801882351F1809192
:10113000590190915A010E94CC15069710F18091A7
:101140004801909149019093510180935001809101
:101150004A0190914B0190935301809352018091E9
:101160004C0190914D0190935501809354018091D1
:101170004E0190914F019093570180935601109228
:1011800058010E944B0581E0DF91CF911F910F9193
:10119000FF90EF90DF90CF90BF90AF909F908F9097
:1011A0007F905F904F90089570E060E09ACFE82FB5
:1011B000F0E0EE0FFF1FE05BFE4F8081918108950C
:1011C00008959093600180935F010895E0915F011D
:1011D000F0916001309721F00190F081E02D0994A9
:1011E00080E00895E0915F01F0916001309721F077
:1011F0000280F381E02D09940895E0915F01F09160
:101200006001309721F00480F581E02D0994089564
:1012100020915D0130915E012817390771F090939C
:101220005E0180935D01E0915F01F0916001309774
:1012300021F00680F781E02D0994089520915B014B
:1012400030915C012817390771F090935C0180930D
:101250005B01E0915F01F0916001309721F0008423
:10126000F185E02D0994089508950C9434090E94A5
:10127000B7150E94AE070C9481165F926F927F9211
:101280008F929F92AF92BF92CF92DF92EF92FF9296
:101290000F931F93CF93DF9300D000D00F92CDB761
:1012A000DEB70E94120892E6A92E91E0B92E10E056
:1012B00000E088248394912C502E802F0E94D70820
:1012C0007C01F501C190D1905F01C816D90609F4DF
:1012D0005DC08091E90181FD0E94E00890E080E01E
:1012E000CE24DF243401082E02C0660C771C0A9439
:1012F000E2F7960126213721232B09F442C0898386
:101300005A82E620F72081E0EF2809F480E08B8301
:101310000E94C0158160782F9D838C8349815A81FA
:101320006B818D810E94F209000F111FF801EE59A7
:10133000FE4F8081918168267926718260820E94A9
:101340002E190E94E608909161018917B1F10E945F
:10135000E608809361010F900F900F900F900F900F
:10136000DF91CF911F910F91FF90EF90DF90CF9081
:10137000BF90AF909F908F907F906F905F900C94F4
:101380004F0501968A30910509F0ACCF0F5F1F4FD2
:101390000430110509F090CF8FEF89838A831B8277
:1013A0000E94C0158160782F9D838C8349815A816A
:1013B0006B818D810E94F209C2CF0F900F900F9028
:1013C0000F900F90DF91CF911F910F91FF90EF90B1
:1013D000DF90CF90BF90AF909F908F907F906F9055
:1013E0005F900895CF93DF93CDB7DEB72B970FB6FD
:1013F000F894DEBF0FBECDBF4F83588769877A87C9
:101400008B871E8285E0FE013796DE0111960190E2
:101410000D928A95E1F749815A816B817C818D819A
:101420009E812B960FB6F894DEBF0FBECDBFDF9125
:10143000CF910C946910882309F4D8C0823871F4D4
:101440000E94E60881FDD2C089E30E940E140E942A
:10145000D81489E30E944B140C94D814833859F49F
:101460000E94E60880FDC2C083E50E940E140E941F
:10147000D81483E5EFCF843859F40E94E60882FD42
:10148000B5C087E40E940E140E94D81487E4E2CF0E
:101490009CEF980F913A18F40E940E14DDCF90E261
:1014A000980F983050F4877091E001C0990F8A9599
:1014B000EAF7892F0E948F14CFCF9BE5980F9330C6
:1014C00070F4853A31F0863A39F083E890E00C9474
:1014D000080981E890E0FBCF82E890E0F8CF98E53A
:1014E000980F953108F082C0883A09F440C0893AD3
:1014F00009F440C08A3A09F440C08B3A09F440C06C
:101500008C3A09F440C08B3B09F440C08C3B09F491
:1015100040C08D3A09F440C0803B09F440C08E3A87
:1015200009F440C08F3A09F440C0813B09F440C03F
:10153000823B09F440C0833B09F440C0843B09F47A
:1015400040C0853B09F440C0863B09F440C0873B5E
:1015500009F440C0883B09F440C0893B09F440C00D
:101560008A3B09F440C090E080E00C941E0982EEB2
:1015700090E0FBCF89EE90E0F8CF8AEE90E0F5CFD7
:1015800085EB90E0F2CF86EB90E0EFCF83EB90E03D
:10159000ECCF84EB90E0E9CF87EB90E0E6CF8CECEA
:1015A00090E0E3CF8DEC90E0E0CF83E891E0DDCFF9
:1015B0008AE891E0DACF82E991E0D7CF84E991E03F
:1015C000D4CF81E292E0D1CF83E292E0CECF84E229
:1015D00092E0CBCF85E292E0C8CF86E292E0C5CF21
:1015E00087E292E0C2CF8AE292E0BFCF08958823DB
:1015F00009F44BC0823871F40E94E60881FF45C0AF
:1016000089E30E940E140E94D81489E30E944B14AF
:101610000C94D814833859F40E94E60880FF35C032
:1016200083E50E940E140E94D81483E5EFCF84381E
:1016300059F40E94E60882FF28C087E40E940E1435
:101640000E94D81487E4E2CF9CEF980F913AF0F211
:1016500090E2980F983050F4877091E001C0990F94
:101660008A95EAF7892F0E949514D2CF9BE5980FAF
:10167000933020F490E080E00C940809885A85317A
:1016800020F490E080E00C941E090895882321F056
:101690000E948F140C94D8140895882321F00E947E
:1016A00095140C94D81408958F929F92AF92BF9284
:1016B000DF92EF92FF920F931F93CF93DF9300D0AF
:1016C00000D00F92CDB7DEB77C016D837983FC012A
:1016D000058102950F70128111110E94AE140E94B3
:1016E0000714D82E882371F01123A1F08D81805E1C
:1016F000883080F082E00E94F1130E94071491E08C
:10170000D82ED926E981E295EF70F0E0E755FD4D3E
:101710000C944522D12CF6CF09810F70F981F07F0E
:1017200011F00295007F1123B1F0002361F08D814B
:10173000805E883018F02D81211109C0802F0E9411
:101740008F140E94D8148D810E941B0A15C0802F0F
:101750000E94A014F6CF8D810E94F70A002361F049
:101760008D81805E883018F03D81311129C0802F35
:101770000E9495140E94D814DD2009F4D3C10E9460
:10178000E41380FDCFC1F70112820E94DE130E9494
:101790002712C7010E94A30D0E94DE130F900F9025
:1017A0000F900F900F90DF91CF911F910F91FF90AD
:1017B000EF90DF90BF90AF909F908F900C94491264
:1017C000802F0E94A614D6CF49814F70B42E598124
:1017D000507F503219F0B29480EFB8228D81882367
:1017E00069F0813029F1112369F1002359F0F701E3
:1017F000858180FFA8CF8F70858304C0112361F09D
:10180000011104C08B2D0E94460BB6CF8B2D0130E9
:10181000D1F70E94C214B0CF011106C00E94C514B6
:101820008B2D0E944D0BA8CF013009F4A5CFF6CF28
:10183000112321F0063008F09FCFE4CF053008F0E7
:101840009BCFEECF002361F38D810E94F70A94CFE6
:10185000898186958695837069F0813009F08CCFF7
:101860008D8199819370111102C090E080E00E94F7
:101870001E0982CF8D8199819370111102C090E071
:1018800080E00E94080978CF8D81112329F00E9401
:101890003C180E94231970CF0E94A418FACF8981A6
:1018A000837009F05FC0111167CF2D8122952695B5
:1018B0002770220F220F8D818F7090E0B0E0A0E0A2
:1018C0004C015D01022E04C0880C991CAA1CBB1C93
:1018D0000A94D2F7FD8160E070E0CB01F4FF0FC005
:1018E0006FE070E080E090E004C0660F771F881F13
:1018F000991F2A95D2F760957095809590952981CA
:101900002695269523702D832230B1F0233019F1CE
:101910009B01AC01282939294A295B2929833A836B
:101920004B835C833D8169817A818B819C813130DD
:10193000B1F00E94B41120CF9B01AC0128293929B4
:101940004A295B2929833A834B835C83CA01B90105
:101950000E94DE1111CF0E94B411C501B4010E9492
:101960008A110ACF8695112311F08981817088230D
:1019700009F402CF2D81229526952770220F220F80
:101980008D818F7090E0B0E0A0E04C015D01022EEF
:1019900004C0880C991CAA1CBB1C0A94D2F73D8178
:1019A00060E070E0CB0134FF0FC06FE070E080E0DA
:1019B00090E004C0660F771F881F991F2A95D2F701
:1019C00060957095809590954981469546954370B0
:1019D0004D834230B1F0433019F19B01AC0128290D
:1019E00039294A295B2929833A834B835C833D81CA
:1019F00069817A818B819C813130B1F00E94BA1269
:101A0000BBCE9B01AC01282939294A295B292983AE
:101A10003A834B835C83CA01B9010E94E412ACCEC5
:101A20000E94BA12C501B4010E949012A5CE3D8158
:101A3000323F09F447C080F4303F79F1313FD9F1AA
:101A4000832F805E8031D0F0112309F456C001113C
:101A50007ACE89818F7133C04D81433FD1F1443FAC
:101A600099F7112309F43FC089818F7189830E94FE
:101A7000271263E089810E94E8137ECE5D815F704A
:101A80005D8389818F71112321F00E9427128D813E
:101A9000BACE0E9449128D81C4CE112341F0053087
:101AA00008F06ACE89818F710E946E1265CE063071
:101AB00008F062CEF7CF89818F71112339F00E942F
:101AC00027125ACE89818F711123C9F30E944912BE
:101AD00053CE112329F089818F710E9412124CCEAE
:101AE0000E94081249CE81E00E94F113023008F4EE
:101AF00043CE82E00E94F1133FCE0111A5CE898131
:101B00008F71E4CF49814F706D81C7010E94F80346
:101B10000E94031131CE49814F706D81C7010E942F
:101B200051052ACE0F900F900F900F900F90DF91DC
:101B3000CF911F910F91FF90EF90DF90BF90AF90EA
:101B40009F908F9008950F931F93CF93DF93EC0195
:101B50008B819C81892B29F08881998189238F3FF2
:101B600029F4DF91CF911F910F910895CE010E942A
:101B70001A048823B1F3688179818A810E94B413A1
:101B80008C010E940E130E947F11B801CE01DF91DB
:101B9000CF911F910F910C94540B0E94AE140E9490
:101BA000BF140E9481140E94D8140E94141A0E942B
:101BB000231990E080E00E94080990E080E00C94F6
:101BC0001E090E949D140C94CD0D0E94A813282F6D
:101BD000892F82958F70903C80F48A30B0F48430E5
:101BE00020F4823090F480E008958630E1F781E0BF
:101BF000203E88F0213FB9F70EC08C3011F08F30B5
:101C000091F793FB882780F9089581E0203F39F010
:101C100018F4203E40F70895243F29F7FCCF08959B
:101C2000CF93DF9300D000D00F92CDB7DEB70F90E7
:101C30000F900F900F900F90DF91CF910895CF9359
:101C4000DF9300D000D000D0CDB7DEB726960FB618
:101C5000F894DEBF0FBECDBFDF91CF9108951F93E3
:101C6000CF93DF93E0916B0116E080916C018E13AE
:101C700004C0DF91CF911F910895CE2FD0E01E9F19
:101C8000F0011124E359FE4F40815181628173813B
:101C9000848195810E941F0EFE013196E770E5CF89
:101CA00040919D0150919E0160919F017091A00112
:101CB0008091A1019091A2010C941F0E1F93CF93CC
:101CC000DF938091A201807FC1F480919F018823DE
:101CD000A1F080916B01C0916C0160919D017091A8
:101CE0009E014091A0015091A101D62FD723DA0186
:101CF000A095B09516E0C81304C0DF91CF911F9155
:101D0000089590E04115510511F0DF3F31F401963F
:101D10008770F1CF2A0F3B1F17C0189FF001199F42
:101D2000F00D1124E359FE4F21812713F0CF2081BC
:101D30002613EDCF22812111EACF2381348124178C
:101D4000350740F3241B350B283C310500F7209163
:101D5000A2012F7020612093A20126E0289FF001AC
:101D6000299FF00D1124EE58FE4F80818F70806105
:101D700080838DE991E00E94A30DDF91CF911F91A7
:101D80000C942F0E9F92AF92BF92CF92DF92EF9260
:101D9000FF920F931F93CF93DF93CDB7DEB72B97AF
:101DA0000FB6F894DEBF0FBECDBF8C0185E0F80101
:101DB000DE01179601900D928A95E1F7D8014C91BA
:101DC00011965C9111971296EC9012978091A00158
:101DD0009091A101009709F46BC120919D01309170
:101DE0009E01632F62236F3F09F462C11396CD9069
:101DF000DC9090909F01992009F4F8C0C816D9068C
:101E000008F43FC0F601E81BF90BCF01FF24F3945F
:101E1000883C910508F0F12C8DE9A82E81E0B82EC0
:101E20008091A201982F907FFF2009F4B7C09111F3
:101E300080C0FE2C35132AC0241328C0E11026C010
:101E40008F7080618093A2010E94500EC5010E9494
:101E5000A30D8091A201D80115968C938F2D2B96FE
:101E60000FB6F894DEBF0FBECDBFDF91CF911F91AB
:101E70000F91FF90EF90DF90CF90BF90AF909F9029
:101E80000895809590958C0D9D1DC0CFCD2829F08B
:101E9000842F85238F3F09F019C180E0B82FB170DE
:101EA000DB2EE0916B0120916C0136E080FD1CC0BF
:101EB000EE20A1F28091A20181608093A201F12C19
:101EC000CDCF8E2F90E03E9FF0011124E359FE4FBD
:101ED0006181651306C06081641303C062816E1165
:101EE000E7CFFC013196E770E213EBCF4F835887C1
:101EF0008F8198850E94A813292F22952F709032E8
:101F000060F0225F2F70223078F49F7051F0F8015A
:101F10009581907F31F4D12C0AC09F7011F08823F5
:101F2000D1F3805E8830B8F3C8010E94A30DFD2C68
:101F300095CF351306C0241304C0D801EE2009F450
:101F40007BC04F8358878F8198850E94E50D882339
:101F500009F4B8C0EE2009F4B5C08091A201803226
:101F600070F020919D0130919E013A8329831B825C
:101F7000DD82CC828E83CE0101960E94A30D86E085
:101F8000F801ADE9B1E001900D928A95E1F70E9468
:101F90005E0E0E94500EFF24F39460CF911113C087
:101FA0007C2DDB86CA866E2D8B850E94100E8DE9F6
:101FB00091E00E94A30D86E0F50111928A95E9F760
:101FC0000E94500E4BCF3513BCCF2413BACFE11073
:101FD000B8CFD80115968C93C8010E94A30D86E056
:101FE000F50111928A95E9F7F92C38CFC816D90670
:101FF00088F1B601681B790BCB01F12C883C910567
:1020000008F047C0FE2CEE2009F45CC0351330C048
:1020100024132EC08091A20180FD21C0982F907FB3
:10202000F1F0D80115968C931597903F39F0982FC1
:10203000907F905F8F70892B15968C93C8010E94BA
:10204000A30D86E0F801ADE9B1E001900D928A950B
:10205000E1F7B6CF809590958C0D9D1DCECF86E093
:10206000F801ADE9B1E001900D928A95E1F7F6CE65
:102070004F8358878F8198850E94E50D81117FCF0E
:102080008091A20181608093A201C8010E94A30DEA
:10209000E5CE7C2DDB86CA866E2D8B850E94100EC8
:1020A00086E0EDE9F1E0DF011D928A95E9F788CF3E
:1020B000EE2041F04F8358878F8198850E94E50D6F
:1020C00081115DCFC8010E94A30D65CF81E08E25EF
:1020D000E5CE1F93CF93DF93CDB7DEB72C970FB626
:1020E000F894DEBF0FBECDBF4F83588769877A87CC
:1020F0008B879C87CE0107960E94C20E882369F0C9
:102100008A859B85892B39F04F815885842F8523BB
:102110008F3F09F071C016E05FC086E0FE01379680
:10212000DE01119601900D928A95E1F78A859B85D3
:10213000892B89F388859F8189238F3F61F32091C3
:102140006C0130E0C90101968770992740916B01BD
:102150004817190671F40E94E10D10926C0110925B
:102160006B0186E0EDE9F1E0DF011D928A95E9F768
:10217000D2CF96E0929FD001939FB00D1124A35926
:10218000BE4FFE01319601900D929A95E1F7809332
:102190006C010E942F0EBFCF819FC0011124835973
:1021A0009E4F0E94C20E8823E9F0E0916B011E9FB2
:1021B000F0011124E359FE4F408151816281738106
:1021C000848195810E941F0E80916B0190E00196A1
:1021D0008770992780936B0180916B0190916C01BE
:1021E0008913DACF2C960FB6F894DEBF0FBECDBFA1
:1021F000DF91CF911F91089569857A858B859C85A4
:102200000E941F0E88CFEF92FF920F931F93CF93E0
:10221000DF938C01892B89F0F12CEE24E394E80103
:102220002196F8018491843709F457C0A0F48230D4
:1022300009F43EC048F48130D1F0DF91CF911F9175
:102240000F91FF90EF9008959CEF980F9037A8F7AB
:102250000E941B0A0AC0853709F44CC09CE7980FFE
:10226000903758F78F770E94F70A8E0116C00E5FDD
:102270001F4FFE01849190E2980F983060F48770B0
:10228000FE2D01C0FF0F8A95EAF78F2F0E94B1142F
:102290000E94D81402C00E941B0A8F2D815008F49E
:1022A000BECFEFE9FFE03197F1F700C00000F6CFB5
:1022B0000E5F1F4FFE01849190E2980F983050F40A
:1022C0008770FE2D01C0FF0F8A95EAF78F2F0E94BD
:1022D000B714DECF0E94F70AE0CF0E5F1F4FFE015A
:1022E000C491C150D0F28FE99FE00197F1F700C08F
:1022F0000000F7CF0E5F1F4FFE01F490CECF089580
:102300006093C0017093C1018093C2019093C30197
:102310000C94CD0DCF93DF9300D000D0CDB7DEB7B6
:1023200069837A838B839C838091C0019091C101E2
:10233000A091C201B091C30129813A814B815C8196
:10234000822B932BA42BB52B8093C0019093C101BA
:10235000A093C201B093C3010F900F900F900F9004
:10236000DF91CF910C94CD0DCF93DF9300D000D0AF
:10237000CDB7DEB769837A838B839C838091C0015C
:102380009091C101A091C201B091C30129813A810C
:102390004B815C8182239323A423B5238093C001C6
:1023A0009093C101A093C201B093C3010F900F900D
:1023B0000F900F90DF91CF910C94CD0DCF93DF93C1
:1023C00000D000D0CDB7DEB769837A838B839C833E
:1023D0008091C0019091C101A091C201B091C3014F
:1023E00029813A814B815C8182279327A427B527D5
:1023F0008093C0019093C101A093C201B093C30127
:102400000F900F900F900F90DF91CF910C94CD0D06
:102410001092BC011092BD011092BE011092BF013A
:102420000C94CD0D41E050E060E070E004C0440F3A
:10243000551F661F771F8A95D2F74093BC015093B2
:10244000BD016093BE017093BF010C94CD0D282F88
:1024500081E090E0A0E0B0E004C0880F991FAA1FBF
:10246000BB1F2A95D2F74091BC015091BD016091EC
:10247000BE017091BF01842B952BA62BB72B8093A7
:10248000BC019093BD01A093BE01B093BF010C9419
:10249000CD0D41E050E060E070E004C0440F551FF6
:1024A000661F771F8A95D2F7409550956095709575
:1024B0008091BC019091BD01A091BE01B091BF017E
:1024C00084239523A623B7238093BC019093BD0159
:1024D000A093BE01B093BF010C94CD0D282F81E0D5
:1024E00090E0A0E0B0E004C0880F991FAA1FBB1FB6
:1024F0002A95D2F74091BC015091BD016091BE0177
:102500007091BF0184279527A627B7278093BC0128
:102510009093BD01A093BE01B093BF010C94CD0D6B
:10252000CF93DF9300D000D0CDB7DEB769837A8335
:102530008B839C838091BC019091BD01A091BE01D1
:10254000B091BF0129813A814B815C81822B932B11
:10255000A42BB52B8093BC019093BD01A093BE0129
:10256000B093BF010F900F900F900F90DF91CF911C
:102570000C94CD0DCF93DF9300D000D0CDB7DEB754
:1025800069837A838B839C838091BC019091BD0188
:10259000A091BE01B091BF0129813A814B815C813C
:1025A00082239323A423B5238093BC019093BD0180
:1025B000A093BE01B093BF010F900F900F900F90AA
:1025C000DF91CF910C94CD0DCF93DF9300D000D04D
:1025D000CDB7DEB769837A838B839C838091BC01FE
:1025E0009091BD01A091BE01B091BF0129813A81B6
:1025F0004B815C8182279327A427B5278093BC0158
:102600009093BD01A093BE01B093BF010F900F90B6
:102610000F900F90DF91CF910C94CD0D0895E82F7E
:102620002AE0929FE00D11248E2F877041E001C0B7
:10263000440F8A95EAF7E695E695E69585E0E89FEA
:10264000F0011124ED55FE4F30E020E070E0519193
:10265000DF011197CB01022E02C0969587950A944F
:10266000E2F7817081958527842385278C932F5FDE
:102670003F4F2530310559F70895E82F2AE0929F02
:10268000E00D11249E2F9770E695E695E69585E07E
:10269000E89FF0011124ED55FE4F50E040E080E04E
:1026A000219130E0092E02C0369527950A94E2F771
:1026B00021703327042E01C0220F0A94EAF7822BDF
:1026C0004F5F5F4F4530510559F70895BF92CF9244
:1026D000DF92EF92FF920F931F93CF93DF938C01C2
:1026E000C090BC01D090BD01E090BE01F090BF0150
:1026F0008091C0019091C101A091C201B091C3012C
:10270000C82AD92AEA2AFB2ACFE1D0E0BC2ED70179
:10271000C6010C2E04C0B695A795979587950A9487
:10272000D2F780FD0EC0219788F7B12C8B2DDF9159
:10273000CF911F910F91FF90EF90DF90CF90BF90BE
:102740000895B8018C2F0E946E05019761F3EECFBA
:10275000CF93DF93D82FC92F0E9466136D2F7C2F44
:10276000DF91CF910C946E051F93CF93DF93162FBB
:10277000D72F90916A01992339F0862F972FDF91F7
:10278000CF911F910C94A813882391F0862F972F37
:102790000E946613C82F682F812F9D2F0E940F1350
:1027A000612F7D2F8C2FDF91CF911F910C946E059F
:1027B000862F972F0E943D13C82FF2CF8091C4011E
:1027C00085958595859508958091C40187700895B4
:1027D00098E0899F90011124622B6093C4010C94AE
:1027E00027129091C401809589238093C401282FDA
:1027F000277061F4282F082E000C330B9217130654
:1028000029F08595859585950C94491208959091A8
:10281000C401977081E009F480E00895909112015D
:102820009923E1F090911A0297FF18C0E82FE695DE
:10283000E695E695EF3139F12091000130910101E3
:10284000E20FF32FF11D877021E030E001C0220F6D
:102850008A95EAF78181822B818308952091000176
:1028600030910101F90132969FEF40E051918517B7
:1028700051F09F3F19F4511101C0942F4F5F4E3119
:10288000A9F79F3F09F40895290F311D97FD3A9547
:10289000F9018283089590911201992301F1909199
:1028A0001A0297FF1CC0E82FE695E695E695EF31F2
:1028B00039F12091000130910101E20FF32FF11D58
:1028C000877021E030E0A90102C0440F551F8A95AE
:1028D000E2F7CA018095918189238183089520912F
:1028E000000130910101F9013296205E3F4F919134
:1028F000891303C0DF0111971C92E217F307B9F7A0
:10290000089581E090E0E0910001F0910101E80F6D
:10291000F91F1082019680329105A9F708959091D0
:10292000E801982B9093E8010895982F9095809155
:10293000E80189238093E80108951092E801089541
:102940009091E701982B9093E7010895982F909527
:102950008091E70189238093E70108951092E701B0
:1029600008959091E601982B9093E6010895982F91
:1029700090958091E60189238093E6010895109255
:10298000E60108958093C50108951092C501089548
:102990002091000130910101F9013196205E3F4FF5
:1029A00080E0919191118F5FE217F307D1F70895BD
:1029B000E0910001F09101018091E8018083E091B4
:1029C0000001F091010180819091E701892B8083C2
:1029D000E0910001F091010180819091E601892B45
:1029E00080839091C501992361F0E0910001F091FD
:1029F00001018081892B80830E94C814811110926B
:102A0000C50180910001909101010C94F2086DEED6
:102A10007EEF90E080E00E947F2260E082E090E024
:102A20000E946D2260E083E090E00E946D2260E0F1
:102A300084E090E00E946D2260E085E090E00C94DC
:102A40006D2290E080E00E9467229C0181E02D3E93
:102A50003E4F09F080E0089582E090E00C945F2200
:102A6000682F82E090E00C946D2283E090E00C945B
:102A70005F22682F83E090E00C946D2284E090E068
:102A80000C945F22682F84E090E00C946D2280917A
:102A90002002843039F11092EA0188E190E020E4CC
:102AA0000FB6F894A895809360000FBE2093600045
:102AB00080E00E944F0583B7817F846083BF83B726
:102AC000816083BF7894889583B78E7F83BF0FB66C
:102AD000F894A895809160008861809360001092BE
:102AE00060000FBE089508950895CF930E94731556
:102AF0000E9412080E947415C0E08C2F0E94D70813
:102B0000892B31F4CF5FC430C1F780E0CF910895B5
:102B100081E0FCCF0E94E10D0E94E6080C944F0575
:102B20001F921FB61F9211248F939F93AF93BF9351
:102B30008091EA01811113C08091160290911702D1
:102B4000A0911802B09119024196A11DB11D809368
:102B5000160290931702A0931802B0931902BF9126
:102B6000AF919F918F911F901FBE1F90189582E08B
:102B700084BD93E095BD9AEF97BD80936E00089554
:102B80002FB7F8948091160290911702A091180225
:102B9000B09119022FBF0895CF92DF92EF92FF926A
:102BA0009C014FB7F8948091160290911702A09162
:102BB0001802B09119024FBF6C017D01EE24FF2471
:102BC000A90170E060E0C416D506E606F70638F005
:102BD000821B930BFF90EF90DF90CF9008950197A9
:102BE000F7CF1F921FB61F9211248F939F93AF931D
:102BF000BF938091160290911702A0911802B09194
:102C000019020196A11DB11D80931602909317021F
:102C1000A0931802B0931902BF91AF919F918F9129
:102C20001F901FBE1F9018950E94081EF8942FEF4A
:102C300087EA91E6215080409040E1F700C0000013
:102C400087E090EBDC018093290290932A02A09305
:102C50002B02B0932C0288E19CE00FB6F894A89563
:102C6000809360000FBE90936000FFCFAF92BF9241
:102C7000CF92DF92EF92FF920F931F93CF93C0E01A
:102C8000AA24A394B12CE82EF12C8C2F0E94D708F3
:102C90006C0110E000E0C501002E02C0880F991FF2
:102CA0000A94E2F78C219D21892B99F0602F7C2FCB
:102CB00080E00E945205E816F90659F481E0CF91B0
:102CC0001F910F91FF90EF90DF90CF90BF90AF904A
:102CD00008950F5F1F4F0A301105E9F6CF5FC4302A
:102CE000A1F680E0ECCFCF93C82F8CE20E9436167D
:102CF000882321F08C2FCF910C94361680E0CF9151
:102D00000895CF93DF9300D000D0CDB7DEB70E94F7
:102D10002115811102C00E94071595E6998308C00C
:102D20000E9412088FE39CE90197F1F700C00000B0
:102D3000A981A150A983A111F3CF89E20E94731642
:102D4000811110C18AE20E94731681110E94071539
:102D500085E00E94731681110E9414160E942C15A2
:102D60008093E90187E00E947316882371F08BE15C
:102D70000E947316882309F4D1C09091E901892F2C
:102D80008D7F91FF82608093E9018091E9010E942B
:102D900030150E943E1590E090931B0280931A021A
:102DA00080EE0E947316882341F090911A02892FB9
:102DB0008E7F90FF816080931A0289E30E947316D0
:102DC000882341F090911A02892F8D7F91FF8260B4
:102DD00080931A0282EE0E947316882341F090912C
:102DE0001A02892F8B7F92FF846080931A0286EEED
:102DF0000E947316882341F090911A02892F877FD1
:102E000093FF886080931A0283EE0E9473168823D2
:102E100041F090911A02892F8F7E94FF80618093F8
:102E20001A0285E30E947316882341F090911A02DA
:102E3000892F8F7D95FF806280931A0281E30E9423
:102E40007316882341F090911A02892F8F7B96FF89
:102E5000806480931A0281E10E947316882341F0F6
:102E600090911A02892F97FB87F9805880931A0254
:102E700080911A020E94421587E20E94731689838C
:102E80008EE10E947316882319F0B981B260B9836C
:102E90008FE10E947316882319F029812460298309
:102EA00080E20E947316882319F0398138603983D3
:102EB00081E20E947316882319F049814061498399
:102EC00082E20E947316882319F059815062598357
:102ED00083E20E947316882319F0898180648983B4
:102EE00084E20E9473168823B1F1998190689983D6
:102EF00089810E9439153981232F30E050E040E06C
:102F000029833A834B835C83CA01B9010F900F90E8
:102F10000F900F90DF91CF910C9480118EE00E9462
:102F20007316882339F09091E901892F8B7F92FFE6
:102F3000846029CF80E10E9473169091E901882373
:102F400029F0892F877F93FF88601DCF892F8E7F7F
:102F500090FF816018CFA981A111CACF0E943515B9
:102F6000282FCBCF0F900F900F900F90DF91CF9124
:102F700008958091ED0180FF12C06091050185E008
:102F8000689FB001112475956795759567956038B0
:102F90007105A8F561157105A1F1862F089581FFCE
:102FA00009C06091050185E0689FB0011124759505
:102FB0006795EDCF6091050182FD0AC08091EE0119
:102FC0008823D1F09091040160910501891728F0C0
:102FD00085E0689FB0011124DACF869FB0011124EB
:102FE00085E0869F9001879F300D1124692F70E046
:102FF000C9010E943122CBCF65E070E0CECF8FE7D0
:10300000089581E008958091ED0180FF0CC06091EA
:10301000030170E075956795759567956115710564
:1030200049F1862F089581FF06C06091030170E089
:1030300075956795F3CF6091030182FD0BC0909168
:10304000EE019923A1F0609102018091030196178E
:1030500038F0682F70E06038710500F38FE708954D
:10306000899FC001112470E00E943122F4CF61E0F9
:1030700070E0D7CF81E00895803F31F40E94B91706
:1030800081958093F1010895813F19F40E94B91749
:10309000F8CF823F31F40E94B91781958093F001F7
:1030A0000895833F19F40E94B917F8CF893F29F496
:1030B0000E9403188093F20108958A3F21F40E9430
:1030C00003188195F7CF8B3F31F40E940318819547
:1030D0008093F30108958C3F19F40E940318F8CFF0
:1030E000843F31F48091EF0181608093EF01089576
:1030F000853F21F48091EF018260F7CF863F21F474
:103100008091EF018460F1CF873F21F48091EF013E
:103110008860EBCF883F21F48091EF018061E5CF9B
:103120008D3F31F48091ED0181608093ED01089530
:103130008E3F21F48091ED018260F7CF8F3FB9F788
:103140008091ED018460F1CF9091F001803F41F4D6
:103150008091F10187FD1092F101992371F008959A
:10316000813F29F48091F1011816ACF3F6CF823F2C
:1031700081F497FFF2CF1092F0018091F1019091CC
:10318000F201892B9091F301892B49F71092EE01FE
:103190000895833F19F4191674F3DFCF893F39F48A
:1031A0008091F2011816CCF61092F201D6CF8A3F28
:1031B00029F48091F20187FFD0CFF6CF8B3F39F40D
:1031C0008091F30187FFC9CF1092F301C6CF8C3FE6
:1031D00029F48091F3011816BCF3BFCF843F31F47A
:1031E0008091EF018E7F8093EF01B7CF853F21F46F
:1031F0008091EF018D7FF7CF863F21F48091EF0121
:103200008B7FF1CF873F21F48091EF01877FEBCF58
:10321000883F21F48091EF018F7EE5CF8D3F31F41F
:103220008091ED018E7F8093ED0197CF8E3F21F449
:103230008091ED018D7FF7CF8F3F09F08ECF809188
:10324000ED018B7FF0CF8FEE91E00E94FD080E9490
:10325000C0159093EC018093EB0108951F93CF93D9
:10326000DF9300D000D000D0CDB7DEB78091EB0166
:103270009091EC010E94CC15AC018091EE0120915F
:10328000060130E0811106C0209107019AE0299FD4
:10329000900111244217530788F02091F001A0916A
:1032A000F101A9831091F201B091F301BE832111C4
:1032B0000FC09A2F912B9B2B09F0B2C026960FB608
:1032C000F894DEBF0FBECDBFDF91CF911F9108955F
:1032D0008F3F19F08F5F8093EE01121624F40E9445
:1032E000B9178093F0018091F00187FF05C00E941B
:1032F000B91781958093F0012981121624F40E9458
:10330000B9178093F1018091F10187FF05C00E94F8
:10331000B91781958093F1018091F001882309F418
:1033200055C03091F1013D83332309F44FC0282F5C
:10333000880F330B440B550B29833A834B835C83F3
:10334000CA01B9010E94382123E333E343E35FE379
:1033500069837A838B839C8369817A818B819C8149
:103360000E949C2169837A838B839C8369817A8103
:103370008B819C810E9400216093F0018D81082E39
:10338000000C990BAA0BBB0B89839A83AB83BC837C
:10339000BC01CD010E94382123E333E343E35FE323
:1033A00069837A838B839C8369817A818B819C81F9
:1033B0000E949C2169837A838B839C8369817A81B3
:1033C0008B819C810E9400216093F101111624F4ED
:1033D0000E9403188093F2018091F20187FF05C0DB
:1033E0000E94031881958093F2019E81191624F49E
:1033F0000E9403188093F3018091F30187FF05C0B9
:103400000E94031881958093F30126960FB6F894D5
:10341000DEBF0FBECDBFDF91CF911F910C9423195A
:103420008F3F09F057CF68CF85E0EFEEF1E0DF0185
:103430001D928A95E9F71092EE011092ED01089520
:10344000809114020895CF93DF9300D00F92CDB7EF
:10345000DEB720912002243019F523E029838A83E6
:103460009B832093E9008FEF9091E800815095FDB8
:1034700006C095ED9A95F1F700008111F5CF809186
:10348000E80085FF0DC050E040E063E070E0CE0151
:1034900001960E94801C8091E8008E778093E8005E
:1034A0000F900F900F90DF91CF910895CF93DF93FE
:1034B00000D00F92CDB7DEB79C01809120028430FE
:1034C00031F582E08983205831093B832A8383E0E8
:1034D0008093E9008FEF9091E800815095FD06C040
:1034E00095ED9A95F1F700008111F5CF8091E800F4
:1034F00085FF0DC050E040E063E070E0CE01019632
:103500000E94801C8091E8008E778093E8000F90E5
:103510000F900F90DF91CF910895209120022430D9
:10352000F1F422E02093E9002FEF3091E8002150E0
:1035300035FD06C035ED3A95F1F700002111F5CFC4
:103540002091E80025FF0BC050E040E065E070E00E
:103550000E94801C8091E8008E778093E800089597
:10356000CF93DF93D82FC92F809120028430F1F4BC
:10357000909112019923E9F090911A0297FF19C0D6
:103580008093E9008FEF9091E800815095FD06C08F
:1035900095E19A95F1F700008111F5CF8091E8004F
:1035A00050E040E060E270E085FD1AC0DF91CF910D
:1035B000089581E08093E9008FEF9091E8008150B9
:1035C00095FD06C095ED9A95F1F700008111F5CFB4
:1035D0008091E80085FFEACF50E040E068E070E0CD
:1035E0008D2F9C2F0E94801C8091E8008E77809305
:1035F000E80080E2ED2FFC2FA4EFB1E001900D92E6
:103600008A95E1F7D3CF80911F02811109C00E94F2
:10361000081E0E94651E8091E20084608093E20093
:10362000089510921F020895089508950C948A1524
:1036300042E061EC81E00E94841D42E061EC82E0A6
:103640000E94841D42E061EC83E00E94841D42E2FE
:1036500061EC84E00C94841D80912202893089F110
:1036600048F4823009F494C0833009F44FC08130AB
:1036700041F008958A3009F47BC08B3009F461C0B1
:10368000089580912102813A09F03FC08091E800BD
:10369000877F8093E8008091250290912602892BF4
:1036A00061F460E284EF91E070E00E94CF1C8091B1
:1036B000E8008B778093E800089560E090E080E078
:1036C000F3CF80912102813201F580912502909102
:1036D0002602009711F00397C1F48091E800877FDC
:1036E0008093E8008091E80082FF0BC08091F10098
:1036F000809314028091E8008B778093E8000C940B
:10370000B81D809120028111EDCF08958091210292
:10371000813AD9F78091250290912602892BA9F749
:103720008091E800877F8093E8008091E80080FF27
:10373000FCCF809112018093F1008091E8008E7798
:10374000DCCF80912102813201F780912502909196
:103750002602892BD1F68091E800877F8093E800CC
:103760000E94B81D80912302809312010C94E10DF8
:1037700080912102813249F68091E800877F809311
:10378000E8000E94B81D80912402809315020895DC
:1037900080912102813A09F0B8CF8091E800877FBB
:1037A0008093E8008091E80080FFFCCF80911502B3
:1037B000C2CF84B7877F84BF0FB6F894A895809155
:1037C0006000886180936000109260000FBE80E806
:1037D00080936100109261000E9435090E94081ECA
:1037E0000E94651E8091E20084608093E2007894DC
:1037F0000E94E5200E94370988E091E00E94E108DC
:1038000080912002853019F00E943D09F9CF0E9475
:10381000471580911E02882399F30E94751588230D
:1038200079F30E946A1CECCF9C01DA01892F992759
:1038300083309105C1F068F48130910509F445C0E9
:10384000029761F48DE690E023EE35E02D933C93F2
:10385000089581329105E1F0829739F190E080E09E
:1038600030E020E0F3CFC9019927213059F08230B0
:10387000910559F0EFEDF5E0892B81F7849190E007
:103880009F01E4CFE7ECF5E0F9CFE3EBF5E0F6CF0D
:10389000643020F7E62FF0E0EE0FFF1FE35DFE4FF0
:1038A0002081318189E090E0D1CF6430B8F670E0BA
:1038B000FB01EE0FFF1FEB5DFE4F208131816F5D3D
:1038C0007E4FFB01808190E0C1CF82E190E020E556
:1038D00036E0BCCF80E189BD82E189BD09B400FE3C
:1038E000FDCF8091D8008F7D8093D8008091E0003B
:1038F00082608093E0008091E00081FDFCCF08951C
:10390000AF92BF92CF92DF92FF920F931F93CF930C
:10391000DF936C01EB018A010E94D71DF82E811103
:1039200023C00115110539F0F80180819181C81B70
:10393000D90BC80ED91EB12CA12C2097A9F08091CB
:10394000E80085FD22C08091E8008E778093E80032
:1039500001151105A1F0F80180819181A80EB91E11
:10396000B182A08285E0F82E8F2DDF91CF911F913B
:103970000F91FF90DF90CF90BF90AF9008950E947D
:10398000D71D8823D1F2F82EEFCFF60181916F0178
:103990008093F1002197FFEFAF1ABF0ACECFFC0151
:1039A000CB0120912702309128022617370790F08B
:1039B000009729F42091E8002E772093E80040E05A
:1039C000009751F4411108C08091E80082FF31C096
:1039D00080E00895C901F3CF209120022223A9F1AC
:1039E0002530A9F12091E80023FD2DC02091E800A9
:1039F00022FDEACF2091E80020FFE2CF3091F300D2
:103A00002091F200009719F02830310558F041E07C
:103A10002830310509F040E02091E8002E7720930E
:103A2000E800CECF41914093F10001972F5F3F4FC7
:103A3000E9CF80912002882341F0853041F08091C8
:103A4000E80083FFC1CF81E0089582E0089583E01C
:103A50000895FC01CB0120912702309128022617FE
:103A6000370790F0009729F42091E8002E772093F3
:103A7000E80040E0009751F4411108C08091E8004F
:103A800082FF32C080E00895C901F3CF2091200267
:103A90002223B1F12530B1F12091E80023FD2EC0A1
:103AA0002091E80022FDEACF2091E80020FFE2CF3C
:103AB0003091F3002091F200009719F02830310581
:103AC00058F041E02830310509F040E02091E8004D
:103AD0002E772093E800CECF44914093F1003196A9
:103AE00001972F5F3F4FE8CF80912002882341F05C
:103AF000853041F08091E80083FFC0CF81E00895D8
:103B000082E0089583E00895982F973028F08F7011
:103B10008093E90081E008959093E900242F762FA7
:103B200050E0981731F07091EC002091ED00509129
:103B3000F00021FD02C09F5FE8CF3091EB003E7F97
:103B40003093EB003091ED003D7F3093ED003091EC
:103B5000EB0031603093EB007093EC002093ED00AC
:103B60005093F0002091EE0027FDE5CF80E008950E
:103B70008091210287FF13C08091E80082FF06C078
:103B80008091E8008B778093E80004C08091200248
:103B90008111F2CF0895809120028823D9F380917A
:103BA000E80080FFF8CF8091E8008E77ECCF20917D
:103BB000E4003091E50095E6A9012091EC00822F08
:103BC000817020FF06C08091E80080FF06C080E081
:103BD00008952091E80022FD1AC0809120028823D8
:103BE00089F0853089F08091EB0085FD0FC0209130
:103BF000E4003091E50042175307F9F29150E1F6E5
:103C000084E0089582E0089583E0089581E00895B6
:103C10000E94761E0E947E1EE0EEF0E080818160B0
:103C20008083E8EDF0E080818F77808319BCA7ED79
:103C3000B0E08C918E7F8C9380818F7E80831092F8
:103C40001F0208950F931F93CF93DF930E94761E58
:103C50000E947E1EC8EDD0E088818F77888388819E
:103C60008068888388818F7D888319BC10922002A8
:103C700010921C0210921E0210921D0200EE10E023
:103C8000F80180818B7F808388818160888342E016
:103C900060E080E00E94841DE1EEF0E080818E7F94
:103CA0008083E2EEF0E080818160808380818860A3
:103CB0008083F80180818E7F808388818061888302
:103CC000DF91CF911F910F910895E8EDF0E0808191
:103CD0008F7E8083E7EDF0E080818160808384E0E7
:103CE00082BF81E080931F020C94221EE8EDF0E079
:103CF00080818E7F80831092E20008951092DA0016
:103D00001092E10008951F920F920FB60F921124A6
:103D10002F933F934F935F936F937F938F939F93D3
:103D2000AF93BF93EF93FF938091E10082FF0BC0AD
:103D30008091E20082FF07C08091E1008B7F809339
:103D4000E1000E94E4208091DA0080FF19C0809198
:103D5000D80080FF15C08091DA008E7F8093DA0052
:103D60008091D90080FF94C080E189BD82E189BD46
:103D700009B400FEFDCF81E0809320020E94031B66
:103D80008091E10080FF19C08091E20080FF15C0A2
:103D90008091E2008E7F8093E2008091E20080615A
:103DA0008093E2008091D80080628093D80019BC93
:103DB00085E0809320020E94151B8091E10084FF22
:103DC00029C08091E20084FF25C080E189BD82E1A5
:103DD00089BD09B400FEFDCF8091D8008F7D80930E
:103DE000D8008091E1008F7E8093E1008091E20015
:103DF0008F7E8093E2008091E20081608093E200F8
:103E000080911C02882309F449C084E08093200239
:103E10000E94161B8091E10083FF29C08091E2007F
:103E200083FF25C08091E100877F8093E10082E0DD
:103E30008093200210921C028091E1008E7F80937B
:103E4000E1008091E2008E7F8093E2008091E200A9
:103E500080618093E20042E060E080E00E94841D87
:103E60008091F00088608093F0000E94141BFF9105
:103E7000EF91BF91AF919F918F917F916F915F91E2
:103E80004F913F912F910F900FBE0F901F9018955B
:103E900019BC109220020E94111B72CF8091E30086
:103EA00087FD02C081E0B2CF83E0B0CF1F920F92B6
:103EB0000FB60F9211242F933F934F935F936F93FD
:103EC0007F938F939F93AF93BF93CF93DF93EF93A2
:103ED000FF93D091E900DF708091EC00C82FC17092
:103EE00080FDC0E81092E9008091F000877F809308
:103EF000F00078940E949A1F1092E9008091F000DF
:103F000088608093F000CD2BCF70C093E900FF91C3
:103F1000EF91DF91CF91BF91AF919F918F917F9161
:103F20006F915F914F913F912F910F900FBE0F9026
:103F30001F9018951F93CF93DF93CDB7DEB7AA9745
:103F40000FB6F894DEBF0FBECDBF81E292E0FC0158
:103F500001962091F100208322E089329207B9F77F
:103F60000E942C1B8091E80083FF16C180912102E2
:103F7000909122029A3008F00FC1E92FF0E0E75447
:103F8000FD4D0C944522803881F0823809F004C13F
:103F9000809125028F708093E9008091EB0085FB72
:103FA000882780F91092E90006C080911D02909147
:103FB0001E02911182609091E800977F9093E80033
:103FC0008093F1001092F1008091E8008E77E0C0BC
:103FD000882309F4CEC0823009F0DEC0809123022C
:103FE0008111D1C0809125028F7009F4D5C08093D2
:103FF000E9002091EB0020FFC6C0933031F480919E
:10400000EB0080628093EB00BEC09091EB0090616A
:104010009093EB0021E030E001C0220F8A95EAF78F
:104020002093EA001092EA008091EB008860EACFCA
:104030008111B2C0109123021F778091E300807834
:10404000812B8093E3008091E800877F8093E800D4
:104050000E94B81D8091E80080FFFCCF8091E300B2
:1040600080688093E30082E0111183E08093200256
:1040700093C08058823008F08FC0809123029091C5
:1040800024028C3D23E09207A1F583E08A838AE233
:1040900089834FB7F894DE01139620E03EE051E2A9
:1040A000E32FF0E050935700E49120FF03C0E29526
:1040B000EF703F5FEF708E2F90E0EA30C0F0C79650
:1040C0008D939D932F5F243159F74FBF8091E80066
:1040D000877F8093E8006AE270E0CE0101960E943B
:1040E000CF1C8091E8008B778093E80055C0C09684
:1040F000E7CFAE014F5F5F4F609125020E94141C15
:10410000BC01892B09F448C08091E800877F809327
:10411000E80089819A810E94291DE3CF8038E1F56A
:104120008091E800877F8093E80080911C02809353
:10413000F1004ACF811130C090912302923060F596
:104140008091E800877F8093E80090931C020E9492
:10415000B81D80911C02882311F084E005C0809175
:10416000E30087FDFACF81E0809320020E94181BB4
:1041700013C080912302813079F481E0933009F0FB
:1041800080E080931E021092E9008091E800877F12
:104190008093E8000E94B81D8091E80083FF0AC068
:1041A0008091E800877F8093E8008091EB00806237
:1041B0008093EB00AA960FB6F894DEBF0FBECDBF7A
:1041C000DF91CF911F9108950895CF9380912002A0
:1041D0008823A1F0C091E900CF709091EC00892F65
:1041E000817090FD80E8C82B1092E9008091E80072
:1041F00083FD0E949A1FCF70C093E900CF9108956C
:104200000E9407216894B1110C94962108950E9490
:104210007B2188F09F5798F0B92F9927B751B0F0BC
:10422000E1F0660F771F881F991F1AF0BA95C9F73A
:1042300014C0B13091F00E949521B1E008950C9422
:104240009521672F782F8827B85F39F0B93FCCF3D5
:10425000869577956795B395D9F73EF490958095B7
:10426000709561957F4F8F4F9F4F0895E89409C0D7
:1042700097FB3EF490958095709561957F4F8F4F99
:104280009F4F9923A9F0F92F96E9BB279395F695AF
:10429000879577956795B795F111F8CFFAF4BB0F2D
:1042A00011F460FF1BC06F5F7F4F8F4F9F4F16C091
:1042B000882311F096E911C0772321F09EE8872F1B
:1042C000762F05C0662371F096E8862F70E060E0D7
:1042D0002AF09A95660F771F881FDAF7880F969550
:1042E000879597F9089557FD9058440F551F59F039
:1042F0005F3F71F04795880F97FB991F61F09F3FD3
:1043000079F087950895121613061406551FF2CFFB
:104310004695F1DF08C0161617061806991FF1CF4B
:1043200086957105610508940895E894BB27662772
:104330007727CB0197F908950E94AF210C94202292
:104340000E94122238F00E94192220F0952311F0C9
:104350000C9409220C940F2211240C9496210E9493
:10436000732170F3959FC1F3950F50E0551F629F25
:10437000F001729FBB27F00DB11D639FAA27F00DBE
:10438000B11DAA1F649F6627B00DA11D661F829FE5
:104390002227B00DA11D621F739FB00DA11D621FCA
:1043A000839FA00D611D221F749F3327A00D611DE7
:1043B000231F849F600D211D822F762F6A2F1124C9
:1043C0009F5750409AF0F1F088234AF0EE0FFF1FFC
:1043D000BB1F661F771F881F91505040A9F79E3F53
:1043E000510580F00C9409220C9496215F3FE4F370
:1043F000983ED4F3869577956795B795F795E795A9
:104400009F5FC1F7FE2B880F911D9695879597F9B1
:10441000089597F99F6780E870E060E008959FEF46
:1044200080EC089500240A9416161706180609064B
:10443000089500240A94121613061406050608951A
:10444000092E0394000C11F4882352F0BB0F40F4A2
:10445000BF2B11F460FF04C06F5F7F4F8F4F9F4FE2
:10446000089597FB072E16F4009407D077FD09D026
:104470000E944B2207FC05D03EF4909581959F4FFA
:104480000895709561957F4F0895EE0FFF1F059079
:10449000F491E02D0994AA1BBB1B51E107C0AA1F90
:1044A000BB1FA617B70710F0A61BB70B881F991FD5
:1044B0005A95A9F780959095BC01CD010895F99979
:1044C000FECF92BD81BDF89A992780B50895A8E1E5
:1044D000B0E042E050E00C948722262FF999FECFFD
:1044E00092BD81BDF89A019700B4021639F01FBA47
:1044F00020BD0FB6F894FA9AF99A0FBE0895019666
:10450000272F0E946E220C946D22DC01CB01FC014E
:10451000F999FECF06C0F2BDE1BDF89A319600B41C
:104520000D9241505040B8F70895F894FFCFBA0467
:10453000C604CA04CE04D204D604DA04DE04E204BB
:10454000E604EA04EE04F204F604FA04FE040205AA
:1045500006058C0B8C0BE40BE40B280C440CBC0BF9
:10456000BC0B4F0CBC0B170D170D820DBC0BBC0BFD
:104570008B0DC31FE81FCC20E81FCC20182039204A
:06458000CC208E209A20E1
:10458600C6012808140A321E201AB01A8D1A561AA5
:10459600231A01323635C69766F0F1F2F3943433B6
:1045A60031404D36391E07D1069B066206F5050ECB
:0645B60006270640060086
:00000001FF
